:100000000C949F000C94B40B0C948D0B0C94C700B3
:100010000C94C7000C94C7000C94C7000C94C70044
:100020000C94C7000C94C7000C94C7000C94C70034
:100030000C94C7000C94C7000C94C7000C94C70024
:100040000C94430B0C94C7000C94C7000C94C7008D
:100050000C94C7000C94C7000C94C7000C94C70004
:100060000C94DB0B0C94C70007634236B79BD8A7F0
:100070001A39685618AEBAAB558C1D3CB7CC5763CD
:10008000BD6DEDFD753EF6177231BF000000803F7B
:1000900008000000BE922449123EABAAAA2ABECD97
:1000A000CCCC4C3E00000080BEABAAAAAA3E000009
:1000B0000000BF000000803F000000000008417801
:1000C000D3BB4387D1133D190E3CC3BD4282AD2B38
:1000D0003E68EC8276BED98FE1A93E4C80EFFFBE30
:1000E00001C4FF7F3F00000000000000000024006A
:1000F00027002A0000000000250028002B0004042F
:1001000004040404040402020202020203030303BF
:10011000030301020408102040800102040810209B
:100120000102040810200000000800020100000382
:1001300004070000000000000000FA0C1011112458
:100140001FBECFEFD8E0DEBFCDBF11E0A0E0B1E031
:10015000E0ECFFE202C005900D92A032B107D9F7A2
:1001600022E0A0E2B1E001C01D92A635B207E1F79E
:1001700010E0CEE9D0E004C02197FE010E94A8164D
:10018000CD39D107C9F70E94270D0C94D3170C94D1
:100190000000982F20911A0281E0213208F043C01C
:1001A0008091F6018111FCCF8091190232E03093E9
:1001B000F6019093F5019FEF9093F4011092F301F3
:1001C0002093F201A9EFB1E0E2EDF1E090E0291314
:1001D00031C01092D1019091D101880F892B809369
:1001E000D1018091D001813049F51092D0018091E8
:1001F000D1018093BB008091BC0083FDF8CF85ECDA
:100200008093BC008091F6018230E1F38091F4018B
:100210008F3FB1F08091F4018032A1F08091F40120
:10022000803391F084E01092F80110921A0210923B
:10023000F70108953D9131939F5FC9CF85EEE0CFDF
:1002400080E0F1CF82E0EFCF83E0EDCF9091F60137
:100250009111FCCF91E09093F6014093F5012FEFBF
:100260002093F4011092F301260F2093F201909352
:10027000D1019091D101880F892B8093D101809178
:10028000D0018130F9F41092D0018091D101809396
:10029000BB008091BC0083FDF8CF85EC8093BC004F
:1002A0008091F6018130E1F38091F301861710F41B
:1002B0006091F301A2EDB1E0E0EBF1E080E08613A4
:1002C00003C0089585EEEACF9D9191938F5FF7CF9C
:1002D0008F929F92AF92BF92CF92DF92EF92FF9256
:1002E0000F931F93CF93DF93EC0180912E028F70B9
:1002F000882E8881807F8829888390902E02992D6E
:10030000907F992E8F70982A988290912F029F77D4
:1003100089818078892B898320912F02221F2227AF
:10032000221F90913002392F330F432F422B292F58
:10033000221F2227221F909131029170990F592F6D
:10034000522B40FB87F98983952F9795992797958D
:10035000842F8695892B8A8351FB992790F98B816D
:100360008E7F892B8B8390913102392F3695209186
:100370003202922F979599279795932B622F669526
:1003800030913302232F279522272795262B692F7B
:10039000660F8170862B8B83822F880F991F992778
:1003A000991F982B9C83221F2227221F8D81807EDC
:1003B0003E71822B832B8D83A12C8AECB82E9AE977
:1003C000C92E2BE3D22EE12CF12C00E010E09A0193
:1003D00040E050E060E070E080E090E00E944E1568
:1003E000AA24AA94EFE7BE2EC12CD12C0E94041699
:1003F000F22E032F142FF52F2C873D874E875F8712
:10040000A4E1B0E00E944315688B798B8A8B9B8BAB
:1004100083E08815D8F0EF8191E0891650F1A9E1C9
:10042000B0E02F2D302F412F5F2F0E944315688B96
:10043000798B8A8B9B8B8AE08E83E160EF838DE7DB
:1004400090E09B878A8789E190E01DC084E0881650
:10045000E9F097E09815A0F5DF91CF911F910F91EA
:10046000FF90EF90DF90CF90BF90AF909F908F90D4
:1004700008958AE08E83E160EF8380E991E09B87B5
:100480008A8784E690E099878887E6CF82E48E8326
:100490008F818E7F8F838DE790E09B878A8780EDA9
:1004A00092E1A3E1B0E08C879D87AE87BF8780E8AB
:1004B00096E9A8E9B0E0888B998BAA8BBB8BCCCF4F
:1004C0008E81807C8A608F738E838F818E7F8F83F5
:1004D00080E293E09B878A8780E991E0998788870B
:1004E0001C861D861E861F86188A198A1A8A1B8AF0
:1004F000892D8F70863019F48CE18E83ADCF8730D3
:1005000009F0AACF8EE2F9CF08950895CF92DF9235
:10051000EF92FF92CF93DF93EC0180914B02909189
:100520004C024FE6C42E42E1D42E43E0E42E40E4D8
:10053000F42E811524E0920771F190F4009709F4EC
:100540005DC05FE6C52E52E1D52E53E8E52E50E49E
:10055000F52E81159240F9F0C12CD12C76011BC0EB
:100560002FE6C22E22E1D22E23E0E22E2FE3F22E3E
:10057000811528E0920779F081152AE09207A9F108
:100580008115964049F73FE6C32E32E1D32E33E87A
:10059000E32E3FE3F32E20914A0260E070E880E012
:1005A00090E004C095958795779567952A95D2F741
:1005B0000E944A129B01AC01C701B6010E94A01122
:1005C0006B017C01BE01DD0F880B990B0E944A1262
:1005D0009B01AC01C701B6010E94D612DF91CF91F9
:1005E000FF90EF90DF90CF9008959FE6C92E92E1A3
:1005F000D92E93E8E92E9EE3F92ECDCF86EAC82EB8
:100600008BE9D82E84ECE82E80E4F82EC4CFCF936B
:10061000DF93EA01DC0111968D919C91DC01ED9153
:10062000FC910280F381E02D0995C817D90729F4C0
:1006300081E00E94C90091E0811190E0892FDF9153
:10064000CF910895089590E0FC01EA5DFE4F24915A
:10065000FC01EE5EFE4F3491FC01E250FF4FE4914D
:10066000EE23C9F0222339F0233001F1A8F4213020
:1006700019F1223029F1F0E0EE0FFF1FEC50FF4F8F
:10068000A591B4918FB7F894EC91611126C0309583
:100690003E233C938FBF08952730A9F02830C9F03E
:1006A000243049F7809180008F7D03C080918000C5
:1006B0008F7780938000DFCF84B58F7784BDDBCFC9
:1006C00084B58F7DFBCF8091B0008F778093B00091
:1006D000D2CF8091B0008F7DF9CF3E2BDACF109230
:1006E000AF011092AE011092F80110921A0210920E
:1006F000F60181E08093F5011092D00161E082E182
:100700000E94230361E083E10E942303E9EBF0E010
:1007100080818E7F808380818D7F808388E4809339
:10072000B80085E48093BC0084E892E09093AD012A
:100730008093AC0185E892E09093AB018093AA018D
:100740000895CF93DF9390E0FC01EE5EFE4F24917D
:1007500082509F4FFC0184918823C9F090E0880F5C
:10076000991FFC01E651FF4FA591B491FC01EC509B
:10077000FF4FC591D49161110DC09FB7F8948C9132
:10078000209582238C938881282328839FBFDF9123
:10079000CF910895623051F49FB7F8943C91822F25
:1007A000809583238C93E8812E2BEFCF8FB7F8941D
:1007B000EC912E2B2C938FBFEACF1F93CF93DF9317
:1007C000182FEB0161E00E94A103209739F460E04B
:1007D000812FDF91CF911F910C942303CF3FD1053F
:1007E00011F461E0F5CFE12FF0E0EA5DFE4FE49116
:1007F000E33031F140F4E130B1F0E230E1F0C03803
:10080000D1057CF7E4CFE73029F1E83059F1E43045
:10081000B1F780918000806280938000D0938B003C
:10082000C0938A0004C084B5806884BDC7BDDF91D1
:10083000CF911F91089584B5806284BDC8BDF7CF64
:1008400080918000806880938000D0938900C0935D
:100850008800EDCF8091B00080688093B000C09395
:10086000B300E5CF8091B00080628093B000C09368
:10087000B400DDCF089585ED8093BC008091BC006D
:1008800084FDFCCF1092F601089520917501260F8A
:100890003327331F21323105ECF42091F601FC019E
:1008A00090E080E0243069F082E00895A091750125
:1008B0002191AC014B5A5E4FA40FB52FB11D2C9363
:1008C0000196861798F380917501680F6093750102
:1008D00080E0089581E008950895E091AF0180914E
:1008E000AE01E81730F4F0E0E055FE4F808190E073
:1008F00008958FEF9FEF08959091AF018091AE0121
:100900002FEF3FEF981748F4E92FF0E0E055FE4F46
:10091000208130E09F5F9093AF01C90108958091DD
:10092000AE019091AF01891B990B0895CF92DF9290
:10093000EF92FF920F931F93CF93DF937C01CB0134
:100940008A012091F701222389F0EB016B01C40E8B
:10095000D51ECC15DD0569F06991D701ED91FC91AB
:100960000190F081E02DC7010995F3CF642F0E941B
:100970004504C801DF91CF911F910F91FF90EF9037
:10098000DF90CF900895CF93DF931F92CDB7DEB75E
:1009900069832091F7012223F9F020911A02203275
:1009A00058F021E030E0FC013383228390E080E0C6
:1009B0000F90DF91CF9108958091F801E82FF0E03A
:1009C000E750FE4F998190838F5F8093F801809369
:1009D0001A0281E090E0ECCF61E0CE0101960E9426
:1009E0004504F7CF81E00C94C900CF93DF93EB016E
:1009F00091E09093F701409319021092F801109240
:100A00001A02682F8BE192E00E94C3046D2F8BE1E4
:100A100092E00E94C3046C2F8BE192E00E94C30419
:100A20008BE192E00E94F20483E290E00197F1F7FB
:100A3000DF91CF91089590E080E00895CF93DF9308
:100A4000EC018B818823A9F089819A81288131E08A
:100A50003093F701209319021092F80110921A02B4
:100A60000E94F20491E0811190E0892FDF91CF91F3
:100A700008950E946F0381E08B83CE010E941E05C2
:100A8000982F8111E1CFF1CFCF93C62F91E09093B2
:100A9000F701609319021092F80110921A02682F60
:100AA0008BE192E00E94C3048BE192E00E94F20489
:100AB00083E290E00197F1F741E062E08C2F0E9421
:100AC00026011092AF018093AE018BE192E00E946B
:100AD0007C04C82F8BE192E00E947C0420E0822BF2
:100AE0009C2BCF910895CF93DF93C5E3D2E068812B
:100AF0006F7780E00E94440548814F77BC0180E019
:100B0000DF91CF910C94F504CF93DF9380934F0244
:100B10008091480290914902DC0114962D913C91FC
:100B20001597232B81F02C9131E03093F70120931E
:100B300019021092F80110921A0241E050E06FE49D
:100B400072E00E940703C0914802D09149028C8153
:100B50009D81029708F141E062E088810E942601B0
:100B60001092AF018093AE018230B1F489819A81F5
:100B7000DC01ED91FC910284F385E02D09958093D1
:100B80004F0289819A81DC01ED91FC910284F38509
:100B9000E02D09958093500280914F029091500270
:100BA000982789279827DF91CF910895482F209182
:100BB0004B0230914C0280914D0290914E02822B5B
:100BC000932B423009F443C0433009F443C0413011
:100BD000D9F183609164906821E020934F02909353
:100BE0005002809351028091480290914902FC0189
:100BF000448155814330510578F030812093F701CD
:100C0000309319021092F80110921A0243E050E05A
:100C10006FE472E00E94070381E00E94840597FF61
:100C2000FBCF80E00E94840520914A02022E02C080
:100C3000969587950A94E2F7222329F08115F8E02A
:100C40009F0708F0906F089583609165C4CF83601B
:100C50009166C1CF83609167BECFDF92EF92FF9222
:100C60000F931F93CF93DF93CDB7DEB764970FB683
:100C7000F894DEBF0FBECDBF90912A029817B9F14C
:100C800090912902981798F1D82E86E0D89EF0010D
:100C9000112480912B02811138C0009127021091FC
:100CA00028020E0F1F1F87E2E82E82E0F82E07525F
:100CB0001240C8018E0D9F1D0E941D11F7018783F0
:100CC000FFEFEF1AFF0A8DE2E81682E0F80689F7D7
:100CD000D0922A02CE0101960E94680184E1FE01B1
:100CE0003196A4E3B2E001900D928A95E1F7649603
:100CF0000FB6F894DEBF0FBECDBFDF91CF911F912D
:100D00000F91FF90EF90DF90089520912C02309189
:100D10002D02E20FF31F86E0AEE2B2E001900D92E9
:100D20008A95E1F7D5CF2F923F924F925F926F92C3
:100D30007F928F929F92AF92BF92CF92DF92EF926B
:100D4000FF920F931F9380E00E942D068091340242
:100D50008F708550833008F094C080E00E942D068B
:100D6000809134028F70843009F066C00E9493062F
:100D700020E43DE043E050E00E940E1549018091DF
:100D8000340282958F7082FD03C080FD0E9473053E
:100D9000809134028F70843009F067C00E949306FE
:100DA00028EC30E040E050E00E940E1529013A01A5
:100DB00020913702269580913802482F4795442785
:100DC0004795982F969580913902382F379533277C
:100DD000379586958F70A42EA22AB32EB92AC82ED5
:100DE000D12CE12CF12C00E010E020E432E44FE0C3
:100DF00050E060E070E080E090E00E94D315B22FF8
:100E0000A32FF42FE52FA30192016B2F7A2F8F2FA1
:100E10009E2F0E94C8141F910F91FF90EF90DF90BA
:100E2000CF90BF90AF909F908F907F906F905F908A
:100E30004F903F902F900895609135026F77809189
:100E40003A0286958695869587700E9444054C01E6
:100E5000809134028F708550833008F090CFA3E0EA
:100E600095948794AA95E1F78ACF20913C0230911E
:100E70003D02D4010E943C152AE030E040E050E001
:100E800093CF609135026F7790913A029295969543
:100E90009695937080913B028170880F880F892B03
:100EA0000E944405409140025091410260914202EB
:100EB00070914302A82E192F110F110BB92EC12EBC
:100EC000D12EE12EF12E012F9A01AB0160E070E0EE
:100ED00080E090E00E944E15E8EEAE2EF3E0BF2ECB
:100EE000C12CD12CE12CF12C00E010E00E94D31594
:100EF000B901CA0190CFFF920F931F93CF93DF9355
:100F0000EC01F62E08811981C8010E941D11F81606
:100F100021F06F2DC8010E942511CE01DF91CF91E4
:100F20001F910F91FF900895EF92FF920F931F93DF
:100F3000CF93DF9300D0CDB7DEB796E0E4E3F2E0E5
:100F4000AEE2B2E001900D929A95E1F796E0899FAA
:100F5000D001112480912B02811128C00091270219
:100F6000109128020A0F1B1F87E2E82E82E0F82E5C
:100F700007521240C8018E0D9F1D9A838983F70185
:100F80006781CE0101960E947B07FFEFEF1AFF0AEF
:100F90008DE2E81682E0F80669F70F900F90DF9176
:100FA000CF911F910F91FF90EF90089580912C02A7
:100FB00090912D02A80FB91F86E0EEE2F2E00190B9
:100FC0000D928A95E1F7E9CFAF92BF92CF92DF926F
:100FD000EF92FF920F931F93CF93909134029F70E3
:100FE0009067909334020E949407809134028F702E
:100FF00009F44AC0843008F0E5C0C0913502CF77CB
:1010000030913702369520913802422F4795442778
:101010004795842F832B322F369520913902422F0A
:10102000479544274795942F932B2695A22FAF7071
:10103000BC018A2F90E02091400230914102409102
:101040004202509143020E94A615E0EAAE2EF6E855
:10105000BF2ECC24C394D12CE12CF12C00E010E065
:101060000E94041659016A017B018C0120E030E4E2
:101070004DE053E060E070E080E090E00E940416F4
:101080004C2FB90185E093C0C0913502CF773091E4
:101090003702369520913802422F479544274795CD
:1010A000842F832B322F369520913902422F47957A
:1010B00044274795942F932B2695A22FAF70BC0100
:1010C0008A2F90E0209140023091410240914202EB
:1010D000509143020E94A615B0EAAB2E16E8B12E3D
:1010E000CC24C394D12CE12CF12C00E010E00E9420
:1010F000041659016A017B018C0120E030E04AE6C8
:1011000058E160E070E080E090E00E9404164C2F0F
:10111000B90185E00E94F50480913702582F569559
:1011200090913802692F679566276795262F252BA2
:10113000592F569590913902692F679566276795C3
:10114000362F352B9695492F4F7050E0C0913502C0
:101150009C2F991F9927991FB0913602AB2FAA0F88
:10116000A92BBB1FBB27BB1F8170880FB82B0E9408
:10117000431528EE33E040E050E00E94EC1460E0BC
:101180002932310548F061E02135310528F063E06E
:10119000213A310508F462E04C2F4F7770E0762F4A
:1011A0006627770F770F770F6F69716280E0CF91B5
:1011B0001F910F91FF90EF90DF90CF90BF90AF9075
:1011C0000C94F504CF911F910F91FF90EF90DF9059
:1011D000CF90BF90AF9008954F925F926F927F92A1
:1011E0008F929F92AF92BF92CF92DF92EF92FF9237
:1011F0000F931F93CF93DF9300D0CDB7DEB77894D2
:101200000E9493060E944A1220E030E04AE754E42C
:101210000E94A0110E9412126B017C01C092510128
:10122000D0925201E0925301F092540180E00E946A
:101230002D06609135026F7780913A0287700E9487
:1012400044058C0180913402982F9F702BEF290F59
:10125000233010F0911105C093E0169507959A95EB
:10126000E1F782958F7082FD03C081FD0E947305B6
:10127000A0913E02B0913F0298010E942D1524E6F4
:1012800030E040E050E00E94EC14B90190E080E0D2
:101290000E94481220E030E04AE754E40E94A01186
:1012A00060934D0170934E0180934F0190935001D4
:1012B000AEE3B8E0A70196010E944315609349018F
:1012C00070934A0180934B0190934C0160914901C6
:1012D00070914A0180914B0190914C01C090A20104
:1012E000D090A301E090A401F090A50120E13EE0A0
:1012F00040E050E00E940E15C21AD30AE40AF50A33
:10130000C092A201D092A301E092A401F092A501A3
:101310006091A1011A821982CE0101960E947B0779
:1013200082E00E94D6050E94860260933401709389
:101330003501809336019093370181E00E94D605F4
:101340000E94860260932C0170932D0180932E01E0
:1013500090932F0180E00E94D6050E948602609340
:10136000240170932501809326019093270183E047
:101370000E94D6050E9486026B017C0120E030E0CD
:1013800040E850E40E9443134B015C0120E030E050
:1013900040E450E4C701B6010E9443132B013C0115
:1013A0002AEB39EC4CE552ECC501B4010E94D6128F
:1013B0004B015C0127ED33E647EB53E4C301B20177
:1013C0000E94D6129B01AC01C501B4010E943411E8
:1013D0004B015C01A7019601C701B6010E94D6121C
:1013E0002BE734E145E654E40E94D6129B01AC01A0
:1013F000C501B4010E9433114B015C0129E23CE2BA
:1014000043E754E4C701B6010E94D6129B01AC0128
:10141000C501B4010E94341123EC35E147E953E4DE
:101420000E9433110E9419126093480180910401B7
:1014300090910501A0910601B091070180934401AC
:1014400090934501A0934601B09347018091A2017A
:101450009091A301A091A401B091A50180934001B6
:1014600090934101A0934201B093430180915101B7
:1014700090915201A0915301B091540180933C018D
:1014800090933D01A0933E01B0933F0180914901AB
:1014900090914A01A0914B01B0914C018093380189
:1014A00090933901A0933A01B0933B0180913401AC
:1014B00090913501A0913601B091370180933001B0
:1014C00090933101A0933201B093330180912C01AC
:1014D00090912D01A0912E01B0912F0180932801B0
:1014E00090932901A0932A01B0932B0180914D0183
:1014F00090914E01A0914F01B09150018093200135
:1015000090932101A0932201B093230181E0809365
:10151000F70184E0809319021092F80110921A02E8
:1015200044E050E064E471E08BE192E00E949604B4
:1015300044E050E060E471E08BE192E00E949604A8
:101540006091A1018BE192E00E94C30444E050E06D
:101550006CE371E08BE192E00E94960444E050E07D
:1015600068E371E08BE192E00E94960444E050E071
:1015700060E371E08BE192E00E94960444E050E069
:1015800068E271E08BE192E00E94960444E050E052
:1015900060E271E08BE192E00E9496046091480164
:1015A0008BE192E00E94C3048BE192E00E94F2047E
:1015B0001A82198263E2CE0101960E947B0784E0C1
:1015C000E82E81E0F82E01E010E01A830983F7018C
:1015D00061917F01CE0101960E947B070F5F1F4F33
:1015E0000530110591F76091A1011A830983CE019D
:1015F00001960E947B0710E080912902181780F560
:10160000812F0E942D06809134028F70853060F406
:1016100060913502813098F06F7786E00E94440532
:10162000887099277C0118C08830C0F46091350219
:101630006F778FE00E94440581709927F3CF6F7711
:1016400082E00E944405827099277C0160913502F6
:101650006F7783E00E944405EF28A9F21F5FCCCF8B
:101660000F900F90DF91CF911F910F91FF90EF900E
:10167000DF90CF90BF90AF909F908F907F906F90B2
:101680005F904F9008951F920F920FB60F92112402
:101690002F933F938F939F93AF93BF9380919D011F
:1016A00090919E01A0919F01B091A00130919C0169
:1016B00023E0230F2D3758F50196A11DB11D20936E
:1016C0009C0180939D0190939E01A0939F01B093F4
:1016D000A0018091980190919901A0919A01B091F7
:1016E0009B010196A11DB11D8093980190939901D2
:1016F000A0939A01B0939B01BF91AF919F918F915D
:101700003F912F910F900FBE0F901F90189526E8D4
:10171000230F0296A11DB11DD2CF1F920F920FB6BB
:101720000F9211242F933F934F935F936F937F9367
:101730008F939F93AF93BF93EF93FF93E091020139
:10174000F09103010995FF91EF91BF91AF919F91A6
:101750008F917F916F915F914F913F912F910F905A
:101760000FBE0F901F9018951F920F920FB60F92F9
:1017700011242F933F934F935F936F937F938F9396
:101780009F93AF93BF93EF93FF93E0910001F0918C
:1017900001010995FF91EF91BF91AF919F918F91B9
:1017A0007F916F915F914F913F912F910F900FBE5D
:1017B0000F901F9018951F920F920FB60F92112441
:1017C0002F933F934F935F936F937F938F939F9349
:1017D000AF93BF93EF93FF938091B900887F8036DA
:1017E00009F44AC0F0F5883209F4A7C018F5803131
:1017F00009F49BC0B8F4882309F4F9C0883009F4CF
:1018000094C0FF91EF91BF91AF919F918F917F9184
:101810006F915F914F913F912F910F900FBE0F905D
:101820001F901895883109F488C0803251F7809351
:10183000F40114C0803409F49DC040F48033B9F33E
:101840008833F9F68093F40185ECB0C0803509F453
:1018500085C0883509F496C0883499F60E943B0407
:10186000D0CF883909F48CC038F5883729F050F486
:10187000883611F0803729F683E08093F6011092C4
:10188000970157C0883809F47BC0803919F0803837
:1018900009F0B7CF80919701803208F071C0E091D4
:1018A000970181E08E0F809397018091BB00F0E05B
:1018B000E958FE4F80833DC0803B39F0E0F4803A28
:1018C00009F479C0883A09F09CCF84E08093F6014E
:1018D0001092760110927501E091AC01F091AD018A
:1018E00009958091750181110FC081E08093750188
:1018F0001092550109C0803C09F4A6CF883C09F438
:10190000A3CF883B09F07DCFE091760181E08E0F77
:1019100080937601F0E0EB5AFE4F80818093BB000C
:10192000909176018091750129C08091D1018093B9
:10193000BB0085EC8093BC0064CF9091F301809153
:10194000F201981758F5E091F30181E08E0F809332
:10195000F301F0E0EE52FE4F8081E9CFE091F30118
:1019600081E08E0F8093F3018091BB00F0E0EE5296
:10197000FE4F80839091F3018091F2019817C8F295
:1019800085E8D8CFE091F30181E08E0F8093F301D9
:101990008091BB00F0E0EE52FE4F80838091F50114
:1019A00081115CCF81E08093D00184EA8093BC00F8
:1019B0001092F60126CF85EC8093BC001092F601C0
:1019C00080919701803230F4E0919701F0E0E9587E
:1019D000FE4F10826091970170E0E091AA01F091B2
:1019E000AB0187E791E00995109297010ACF109219
:1019F000F40134CFCF93DF93EBE1F2E01382128254
:101A000088EE93E0A0E0B0E084839583A683B7835B
:101A100082E191E091838083E8E4F2E01282148213
:101A2000138280E890E096838583C7E2D2E0198232
:101A300018821A828FEF8B8381E08C8386E090E09E
:101A40000E94AE169E838D83DF91CF910895CF9330
:101A5000DF93CDB7DEB764970FB6F894DEBF0FBE45
:101A6000CDBF789484B5826084BD84B5816084BD27
:101A700085B5826085BD85B5816085BD80916E002C
:101A8000816080936E00109281008091810082605D
:101A9000809381008091810081608093810080919A
:101AA00080008160809380008091B1008460809389
:101AB000B1008091B00081608093B00080917A0085
:101AC000846080937A0080917A00826080937A00AB
:101AD00080917A00816080937A0080917A0080689A
:101AE00080937A001092C10090E080E00E941D1166
:101AF000833209F00DC181E090E00E941D118093B6
:101B0000040182E090E00E941D118093050183E0B2
:101B100090E00E941D118093060184E090E00E94F5
:101B20001D118093070185E090E00E941D118093B4
:101B3000A1018090040190900501A0900601B09051
:101B400007016091A10170E090E080E00E944A12DC
:101B500020E030E048E453E40E94A0116B017C01D6
:101B6000C501B4010E944A129B01AC01C701B60134
:101B70000E94D6120E9412126093A2017093A301D8
:101B80008093A4019093A50161E08BE00E94A103E2
:101B900061E08AE00E94A10361E089E00E94A10364
:101BA00061E086E00E94A10361E085E00E94A1035C
:101BB00060E08EE00E94A10362E082E00E94A10347
:101BC00062E083E00E94A10382E293E0909301012E
:101BD00080930001809169008C7F8260809369000E
:101BE000E89A8CEE98E09093030180930201809133
:101BF0006900837F886080936900E99A61E089E0E9
:101C00000E94230386E090E00E94AE168C0188E4D7
:101C1000F80180838BE192E092838183138260E2FA
:101C2000E62EF12CF582E4821093490200934802DB
:101C30000E946F0381E0F8018383C8010E941E05A2
:101C4000F0922802E09227028091290281110AC1B4
:101C50000E946F0330E4F32EEE24E39440E8D42E88
:101C60005EE3C52E05EA10E0E092F701F09219025A
:101C70001092F80110921A028BE192E00E94F20495
:101C800081111DC080912902853AC8F46F2D80E032
:101C90000E9444055C014F2D60E070E880E00E94E6
:101CA000F5046F2D80E00E9444059C018115904849
:101CB00009F042C04F2DB50180E00E94F504F39475
:101CC000F0E5FF12D1CF8FEF80932A0210E08091D0
:101CD0002902181708F0F0C0812F0E942D0660918C
:101CE00035026F7780E00E944405209134022F7006
:101CF00009F4D2C0283008F0D3C08F739E7F213002
:101D000021F02550233008F0D4C0806C9160C8C009
:101D10008091040190910501A0910601B091070105
:101D20008093A2019093A301A093A401B093A50175
:101D300088EC8093A10128CF2F3989E3380709F077
:101D400064C080912E02807F80932E0280912E02AB
:101D50008F70883009F4B3CF8F2D8F7780932F0247
:101D600085E080933002D0923102C092320280919D
:101D70003302807E80933302CE0101960E94680177
:101D800084E1FE013196A4E3B2E001900D928A95C0
:101D9000E1F780912E028F70853009F060C080914C
:101DA0003402807F856080933402809129020E94F2
:101DB000E4078091290290E00196B8010E94D814AE
:101DC0008093290290913402907F96609093340220
:101DD0000E94E4078091290290E00196B8010E94D8
:101DE000D8148093290290913402907F9760909349
:101DF00034020E94E4078091290290E00196B80124
:101E00000E94D814809329025ACF2732E1E43E077A
:101E1000B1F46F2D8FEF0E9444059C0190912E022A
:101E2000907F2036F2E23F0721F4916090932E02DA
:101E30008DCF232B11F09260F9CF9360F7CF909163
:101E40002E02907F273281E6380711F49460EECF9E
:101E50002732314711F49560E9CF9860E7CF809140
:101E60002902C7CF8FEF0E942D06809135028F7710
:101E70008093350285E08093360280E880933702B4
:101E80008EE38093380280913902807E80933902FC
:101E90008FEF0E94E40717CF8F77987F8068956057
:101EA000409135024F77BC0180E00E94F5041F5F2E
:101EB0000ECF80689360F4CF10E08091290218174C
:101EC000E0F4812F0E942D06609135026F7780E04B
:101ED0000E944405209134022F7021F0283020F414
:101EE000886302C0877C8865409135024F77BC01CA
:101EF00080E00E94F5041F5FE0CF10E0809129028E
:101F00001817E8F4812F0E942D06609135026F7733
:101F100080E00E944405209134022F7029F028307F
:101F200028F4917F986002C0886F976040913502D5
:101F30004F77BC0180E00E94F5041F5FDFCF10E007
:101F400080912902181710F5812F0E942D066091AB
:101F500035026F7780E00E944405887F7C01809184
:101F600034028F70806780933402812F0E9494071F
:101F7000409135024F778091340282958F70B7017E
:101F8000682B80E00E94F5041F5FDACF10E080919B
:101F90002902181708F42AC190E4D92E20E0E22E75
:101FA00020E0F22E2FB7F89480919D0190919E0130
:101FB000A0919F01B091A0012FBF4091A601509127
:101FC000A7016091A8017091A901841B950BA60B34
:101FD000B70B81319742A105B105D8F12FB7F8941D
:101FE00080919D0190919E01A0919F01B091A001CF
:101FF0002FBF8093A6019093A701A093A801B0934F
:10200000A9016091A2017091A3018091A401909116
:10201000A501409004015090050160900601709068
:1020200007010E944A124B015C01C301B2010E94E8
:102030004A129B01AC01C501B4010E94A01120E02D
:1020400030E048E453E40E94D6120E9419126093D3
:10205000A1018FB7F8948FBFD0927C0080917A0055
:10206000806480937A0080917A0086FDFCCF809115
:10207000780000917900102F082F17FF02C00D5F24
:102080001F4F159507951595079511950195110900
:102090001C5F8091A1018091A1018431A0F4B8015D
:1020A00085E00E94DD0360E086E00E94230360E09B
:1020B00089E00E94230360E08AE00E94230360E03D
:1020C0008BE00E9423038091A1018431C0F08091B4
:1020D000A1018C33A0F4B80185E00E94DD0360E02B
:1020E00086E00E94230360E089E00E94230360E011
:1020F0008AE00E94230360E08BE00E94230380912A
:10210000A1018C33C0F08091A1018436A0F4B80104
:1021100085E00E94DD03B80186E00E94DD0360E0F7
:1021200089E00E94230360E08AE00E94230360E0CC
:102130008BE00E9423038091A1018436C0F080913E
:10214000A1018C38A0F4B80185E00E94DD03B8013C
:1021500086E00E94DD03B80189E00E94DD0360E0B3
:102160008AE00E94230360E08BE00E9423038091B9
:10217000A1018C38C0F08091A101843BA0F4B8018A
:1021800085E00E94DD03B80186E00E94DD03B8010E
:1021900089E00E94DD03B8018AE00E94DD0360E06F
:1021A0008BE00E9423038091A101843BC0F08091C9
:1021B000A101893CA0F4B80185E00E94DD03B801CB
:1021C00086E00E94DD03B80189E00E94DD03B801CA
:1021D0008AE00E94DD03B8018BE00E94DD03E11478
:1021E000F10409F4DFCE0E940000DCCE812F0E94B2
:1021F0002D06809134028F708150843078F4609184
:1022000035026F7786E00E94440593704091350255
:102210004F77BC01746086E00E94F5041F5FB7CE63
:1022200080912B02882341F080912C0290912D0205
:10223000009711F00C944A170895F999FECF92BDBA
:1022400081BDF89A992780B50895262FF999FECF78
:102250001FBA92BD81BD20BD0FB6F894FA9AF99AC3
:102260000FBE019608955058BB27AA270E944B1114
:102270000C949C120E948E1238F00E94951220F04D
:1022800039F49F3F19F426F40C948B120EF4E09568
:10229000E7FB0C948512E92F0E94AD1258F3BA1790
:1022A000620773078407950720F079F4A6F50C946C
:1022B000CF120EF4E0950B2EBA2FA02D0B01B90111
:1022C00090010C01CA01A0011124FF27591B99F0AC
:1022D000593F50F4503E68F11A16F040A22F232FB8
:1022E000342F4427585FF3CF469537952795A79508
:1022F000F0405395C9F77EF41F16BA0B620B730BAF
:10230000840BBAF09150A1F0FF0FBB1F661F771F1F
:10231000881FC2F70EC0BA0F621F731F841F48F4D4
:10232000879577956795B795F7959E3F08F0B0CF5D
:102330009395880F08F09927EE0F97958795089544
:102340000E94B4110C949C120E94951258F00E94A5
:102350008E1240F029F45F3F29F00C948512511140
:102360000C94D0120C948B120E94AD1268F3992336
:10237000B1F3552391F3951B550BBB27AA27621781
:102380007307840738F09F5F5F4F220F331F441F8E
:10239000AA1FA9F335D00E2E3AF0E0E832D09150C2
:1023A0005040E695001CCAF72BD0FE2F29D0660FAF
:1023B000771F881FBB1F261737074807AB07B0E8F2
:1023C00009F0BB0B802DBF01FF2793585F4F3AF0F8
:1023D0009E3F510578F00C9485120C94D0125F3F0B
:1023E000E4F3983ED4F3869577956795B795F7957E
:1023F0009F5FC9F7880F911D9695879597F9089566
:10240000E1E0660F771F881FBB1F62177307840701
:10241000BA0720F0621B730B840BBA0BEE1F88F710
:10242000E09508950E9419126894B1110C94D0128D
:1024300008950E94B51288F09F5798F0B92F9927F8
:10244000B751B0F0E1F0660F771F881F991F1AF09F
:10245000BA95C9F714C0B13091F00E94CF12B1E023
:1024600008950C94CF12672F782F8827B85F39F022
:10247000B93FCCF3869577956795B395D9F73EF438
:1024800090958095709561957F4F8F4F9F4F0895E0
:10249000E89409C097FB3EF49095809570956195FE
:1024A0007F4F8F4F9F4F9923A9F0F92F96E9BB27B4
:1024B0009395F695879577956795B795F111F8CF30
:1024C000FAF4BB0F11F460FF1BC06F5F7F4F8F4F9B
:1024D0009F4F16C0882311F096E911C0772321F091
:1024E0009EE8872F762F05C0662371F096E8862F29
:1024F00070E060E02AF09A95660F771F881FDAF780
:10250000880F9695879597F9089597F99F6780E8C2
:1025100070E060E008959FEF80EC089500240A9435
:102520001616170618060906089500240A941216AE
:102530001306140605060895092E0394000C11F4E1
:10254000882352F0BB0F40F4BF2B11F460FF04C08E
:102550006F5F7F4F8F4F9F4F089557FD9058440FE7
:10256000551F59F05F3F71F04795880F97FB991FF2
:1025700061F09F3F79F087950895121613061406AF
:10258000551FF2CF4695F1DF08C01616170618063C
:10259000991FF1CF86957105610508940895E89417
:1025A000BB2766277727CB0197F908950E94E91288
:1025B0000C949C120E948E1238F00E94951220F00A
:1025C000952311F00C9485120C948B1211240C9409
:1025D000D0120E94AD1270F3959FC1F3950F50E099
:1025E000551F629FF001729FBB27F00DB11D639FC5
:1025F000AA27F00DB11DAA1F649F6627B00DA11D6B
:10260000661F829F2227B00DA11D621F739FB00D10
:10261000A11D621F839FA00D611D221F749F332780
:10262000A00D611D231F849F600D211D822F762F19
:102630006A2F11249F5750409AF0F1F088234AF0F6
:10264000EE0FFF1FBB1F661F771F881F9150504062
:10265000A9F79E3F510580F00C9485120C94D0127E
:102660005F3FE4F3983ED4F3869577956795B795E9
:10267000F795E7959F5FC1F7FE2B880F911D969503
:10268000879597F90895FA01EE0FFF1F30962105FF
:102690003105A1F16115710561F48038BFE39B0735
:1026A00049F168949038810561F08038BFEF9B074D
:1026B00041F099234AF5FF3FE1053105210519F164
:1026C000E8940894E795D901AA2329F4AB2FBE2FEB
:1026D000F85FD0F310C0FF5F70F4A695E0F7F7390C
:1026E00050F019F0FF3A38F49F779F930DD00F9078
:1026F00007FC9058089546F00C948B1260E070E04F
:1027000080E89FE308954FE79F775F934F933F9350
:102710002F930E943E142F913F914F915F910E9401
:10272000D6120C949B1329F416F00C9485120C9479
:10273000CF120C948B120E94B512A8F39638A0F712
:1027400007F80F92E8942BE33AEA48EB5FE70E9420
:10275000EC120F920F920F924DB75EB70F920E943C
:102760008614E8E6F0E00E94CD134F915F91EF915F
:10277000FF91E595EE1FFF1F49F0FE57E0684427E3
:10278000EE0F441FFA95E1F74195550B0E94001496
:102790000F9007FE0C94F4130895DF93CF931F93CB
:1027A0000F93FF92EF92DF927B018C01689406C039
:1027B000DA2EEF010E94E912FE01E894A59125911D
:1027C000359145915591A6F3EF010E944B11FE0101
:1027D0009701A801DA9469F7DF90EF90FF900F91CD
:1027E0001F91CF91DF9108959B01AC0160E070E0F3
:1027F00080E89FE30C94A0110C9485120C94BA14F9
:102800000E94B512D8F39923C9F3940F511DA3F375
:102810009150504094F059F0882332F0660F771FA2
:10282000881F91505040C1F79E3F51052CF7880FEB
:10283000911D9695879597F908955F3FACF0983E66
:102840009CF0BB27869577956795B79508F4B1609E
:102850009395C1F7BB0F58F711F460FFE8CF6F5F96
:102860007F4F8F4F9F4FE3CF0C94D01216F00C94F4
:10287000BA140C948B1268940C9485120E94B512B1
:10288000A8F39923C1F3AEF3DF93CF931F930F9374
:10289000FF92C92FDD2788232AF02197660F771F23
:1028A000881FDAF720E030E040E85FEB9FE38839EB
:1028B00020F0803E38F021968F770E943411E0E9B5
:1028C000F0E004C00E943411EDEBF0E00E94CD1363
:1028D0008B01BE01EC01FB2E6F5771097595771FB7
:1028E000880B990B0E944A1228E132E741E35FE32B
:1028F0000E94E912AF2D9801AE01FF900F911F9138
:10290000CF91DF910E944B110C949C12FA01DC01D3
:10291000AA0FBB1F9B01AC01BF5728F42227332706
:102920004427507820C0B75190F4AB2F002446952F
:1029300037952795011CA395D2F3002071F0220F43
:10294000331F441FB395DAF30ED00C94331161306A
:102950007105A0E88A07B94630F49B01AC016627EF
:10296000772788279078309621F02083318342831F
:10297000538308959F3F31F0915020F487957795C8
:102980006795B795880F911D9695879597F9089546
:10299000DB018F939F930E944315BF91AF91A29F3C
:1029A000800D911DA39F900DB29F900D112408954D
:1029B000AA1BBB1B51E107C0AA1FBB1FA617B70765
:1029C00010F0A61BB70B881F991F5A95A9F7809581
:1029D0009095BC01CD010895A1E21A2EAA1BBB1B44
:1029E000FD010DC0AA1FBB1FEE1FFF1FA217B307DB
:1029F000E407F50720F0A21BB30BE40BF50B661FF1
:102A0000771F881F991F1A9469F7609570958095B4
:102A100090959B01AC01BD01CF010895052E97FB58
:102A20001EF400940E94251557FD07D00E94EC1457
:102A300007FC03D04EF40C94251550954095309525
:102A400021953F4F4F4F5F4F08959095809570951A
:102A500061957F4F8F4F9F4F0895A29FB001B39F05
:102A6000C001A39F700D811D1124911DB29F700D97
:102A7000811D1124911D08950E942D15B7FF089501
:102A8000821B930B08950E942D15A59F900DB49F56
:102A9000900DA49F800D911D11240895DF93CF9375
:102AA0001F930F939A9DF02D219FF00D8B9DF00D9C
:102AB0008A9DE02DF10D039FF00D029FE00DF11DA9
:102AC0004E9DE00DF11D5E9DF00D4F9DF00D7F932D
:102AD0006F93BF92AF925F934F93D5010E942D15D4
:102AE0008B01AC01D7010E942D15EB01E80FF91FF6
:102AF000D6010E949D152F913F91D6010E942D1560
:102B0000C60FD71FE81FF91FAF91BF910E949D15F7
:102B10002F913F910E942D15C60FD71FE81FF91F57
:102B2000D6010E942D15E60FF71F9801BE01CF01B7
:102B30000F911F91CF91DF9108950E942D15460F9F
:102B4000571FC81FD91F08F431960895E894DF93E2
:102B5000CF93FC01DB010E942D157F936F93E90158
:102B60009A01AC01BF93AF933F932F93DF010E9473
:102B70002D1526F46C1B7D0B820B930B9E01EB0134
:102B8000FC010E949D15AF91BF912F913F910E9432
:102B90009D15BE01CF01F9012F913F91CF91DF919A
:102BA0000895689401C0E894F92FF12B12F00C9469
:102BB0000516A0E0B0E0EFEDF5E10C947716092ED4
:102BC000059422F40E946116112392F4F0E80F2676
:102BD000FFEFE094F09400951095B094C094D094D9
:102BE000A194BF0ACF0ADF0AEF0AFF0A0F0B1F0BDF
:102BF0000E94101607FC0E946116CDB7DEB7ECE00C
:102C00000C949316689401C0E8948F929F92CF938E
:102C1000DF930E941016DF91CF919F908F900895BF
:102C200088249924F401E401B0E49F93AA279A151B
:102C30008B049C04ED05FE05CF05D007A10798F491
:102C4000AD2FDC2FCF2FFE2FE92D982C892E982F1A
:102C5000872F762F652F542F432F322F2227B850DE
:102C600031F7BF9127C01B2EBF91BB27220F331F07
:102C7000441F551F661F771F881F991F881C991CAA
:102C8000EE1FFF1FCC1FDD1FAA1FBB1F8A149B0452
:102C9000EC05FD05CE05DF05A007B10748F08A1851
:102CA0009B08EC09FD09CE09DF09A00BB10B2160DF
:102CB0001A94E1F62EF49401AF01BE01CD01000C8F
:102CC00008956095709580959095309540955095B4
:102CD00021953F4F4F4F5F4F6F4F7F4F8F4F9F4F0C
:102CE00008952F923F924F925F926F927F928F92B0
:102CF0009F92AF92BF92CF92DF92EF92FF920F938B
:102D00001F93CF93DF93CDB7DEB7CA1BDB0B0FB694
:102D1000F894DEBF0FBECDBF09942A883988488851
:102D20005F846E847D848C849B84AA84B984C884E7
:102D3000DF80EE80FD800C811B81AA81B981CE0FDE
:102D4000D11D0FB6F894DEBF0FBECDBFED010895C3
:102D5000EE0FFF1F0590F491E02D09940F931F9340
:102D6000CF93DF938230910510F482E090E0E09100
:102D70005402F091550230E020E0B0E0A0E030973E
:102D800099F42115310509F44AC0281B390B243068
:102D90003105D8F58A819B816115710589F1FB01A7
:102DA00093838283FE0111C040815181028113818E
:102DB00048175907E0F04817590799F4109761F040
:102DC00012960C93129713961C933296CF01DF91B3
:102DD000CF911F910F9108950093540210935502C3
:102DE000F4CF2115310551F04217530738F0A901EE
:102DF000DB019A01BD01DF01F801C1CFEF01F9CF7D
:102E00009093550280935402CDCFFE01E20FF31F41
:102E1000819391932250310939832883D7CF209110
:102E2000520230915302232B41F420910A01309138
:102E30000B013093530220935202209108013091EC
:102E400009012115310541F42DB73EB740910C0120
:102E500050910D01241B350BE0915202F091530269
:102E6000E217F307A0F42E1B3F0B2817390778F061
:102E7000AC014E5F5F4F2417350748F04E0F5F1FC0
:102E80005093530240935202819391939FCFF0E06D
:102E9000E0E09CCFCF93DF930097E9F0FC013297FD
:102EA00013821282A0915402B0915502ED0130E0DC
:102EB00020E01097A1F420813181820F931F20918F
:102EC0005202309153022817390709F061C0F0937C
:102ED0005302E0935202DF91CF910895EA01CE1799
:102EE000DF07E8F54A815B819E0141155105B1F785
:102EF000E901FB83EA8349915991C40FD51FEC176F
:102F0000FD0761F4808191810296840F951FE9018C
:102F100099838883828193819B838A83F0E0E0E0B8
:102F200012968D919C9113970097B9F52D913C9134
:102F30001197CD010296820F931F2091520230917A
:102F400053022817390739F6309751F51092550278
:102F500010925402B0935302A0935202BCCFD38379
:102F6000C28340815181840F951FC817D90761F42E
:102F70004E5F5F4F88819981480F591F518340836D
:102F80008A819B81938382832115310509F0B0CF1B
:102F9000F0935502E09354029ECFFD01DC01C0CFB7
:102FA00013821282D7CF10E0CEE9D0E004C0FE0138
:102FB0000E94A8162196CF39D107C9F7F894FFCF00
:102FC0003A043A0480841E0000005602800000008B
:102FD0000000C30496041B056C048F047C046D047C
:00000001FF
